:020000040000FA
:020000004C288A
:080008004C288C0081018316D5
:100010000313C030810508008C008101831603138F
:10002000C030810501308104831203130B110B1DB5
:1000300017288C0B162808008E00E13086050E0D5F
:100040001E398604080086132628861706138F009B
:100050000F080F0E1C2033200F081C203320E13026
:1000600086058613080001300C20861600008612D3
:1000700001300C2008001414120893000830950079
:100080003030931B31302520930D950B4028141CE4
:100090000800141011083D2883160313013086054B
:1000A00083120313861206138613E130860504308B
:1000B0000C2003301C20332001300C2008301C2081
:1000C000332001300C2002301C20332001300C2062
:1000D000283023200C3023200130232008300C202E
:1000E00092019101823023204C302520433025207D
:1000F000443025206230252031302520363025201F
:100100002D302520543025206530252073302520C2
:10011000743025203A302520C03023203B20910F19
:0A0120009228920A40300C208C282F
:02400E00F13F80
:00000001FF
